:020000040800F2
:10000000700E002059470008432A00088B2B000877
:10001000472C0008772C0008A72C000800000000DF
:100020000000000000000000000000005F31000838
:10003000C7330008000000001B47000827470008DE
:10004000A5470008A7470008A947000800000000CE
:1000500000000000AB470008A5190008E1190008DE
:10006000AD47000800000000AF470008B147000896
:10007000B347000800000000773F0008B5470008BC
:10008000B7470008B947000800000000BB47000858
:10009000BD47000800000000000000000000000054
:1000A000000000000000000000000000BF47000842
:1000B000C1470008C3470008C5470008C7470008F4
:1000C000002204E00B78D2B28354491C521C0B78F6
:1000D000002BF7D11000C0B2704700002DE9FE4F91
:1000E0000400A4B2012C0DD1DFF8E0ADDFF8E01D73
:1000F0000988891E9AF80020FF2A05D102259AF85E
:1001000003B004E001F0D8BA00259AF801B05FFA14
:100110008BFB5A46032A13D0062A00F09782082A3E
:1001200000F0E187102A00F04185112A00F0F787DE
:100130002B2A01F048805C2A01F06C8201F07EBA23
:100140009AF80000002801F0B78200200090ADB2BC
:100150000AEB050080788DF80100ADB20AEB0500CE
:10016000C0788DF80000ADB20AEB050000798DF87B
:100170000500ADB20AEB050040798DF80400BDF82A
:10018000040015EB4000461D9AF80000DFF8041E3D
:100190000870ADB2002D09D09AF80100DFF8F41D07
:1001A00048709AF80200DFF8EC1D88700098B0F5EE
:1001B0008060FF2800F21582BDF80400812880F2DB
:1001C0001082BDF80400002800F00B820098BDF8F2
:1001D00004100818B0F5A06F00F20382DFF8B40D28
:1001E000ADB2284480F801B09DF804004000DFF86B
:1001F000A41DADB229448870009F5FF0000819E08B
:1002000000200090DFF88C0DADB21FFA88F815EBD6
:10021000480108449DF800100171DFF8780DADB277
:100220001FFA88F815EB480108449DF80110C170C9
:1002300018F101084046BDF8041080B2884280F0F1
:10024000AA811FFA88F818EB07004FF48061401A62
:1002500041D0401E54D0401E55D0401E68D0401E94
:100260007BD0401E00F08E80401E00F0A080401E1B
:1002700000F0B280401E00F0C480401E00F0C98033
:10028000401E00F0CE80401E00F0D080401E00F0E6
:10029000EE80401E00F0F680401E00F0FE80401E02
:1002A00000F00681401E00F00E81401E00F0168115
:1002B000401E00F03481401E00F03C81401E00F0E2
:1002C0004481401E00F04C81401E00F054811338E0
:1002D00000F05C8194E7002000905FF0000908E0E6
:1002E0000098DFF8B41C31F819100818009019F1C3
:1002F0000109B9F1040FF3D300988008009081E759
:10030000002000907EE7002000905FF0000908E0E8
:100310000098DFF8881C31F819100818009019F1BE
:100320000109B9F1040FF3D300988008009069E740
:10033000002000905FF0000908E00098DFF8601CE2
:1003400031F819100818009019F10109B9F1040FDA
:10035000F3D300988008009054E7002000905FF0ED
:10036000000908E00098DFF83C1C31F81910081863
:10037000009019F10109B9F1040FF3D30098800836
:1003800000903FE7002000905FF0000908E000982F
:10039000DFF8141C31F819100818009019F1010940
:1003A000B9F1040FF3D30098800800902AE70020E9
:1003B00000905FF0000908E00098DFF8F01B31F8CA
:1003C00019100818009019F10109B9F1040FF3D3BD
:1003D00000988008009015E7002000905FF0000969
:1003E00008E00098DFF8C81B31F8191008180090D1
:1003F00019F10109B9F1040FF3D3009880080090B6
:1004000000E700200090DFF8AC0B00788DF80100C9
:10041000F8E600200090DFF8A00B00788DF80100CE
:10042000F0E6DFF8980B00680090EBE6DFF8900B41
:1004300000684FF6FB710840DFF8841B08600C2150
:10044000DFF8800B01F03CFADFF8740B006850F025
:100450000C00DFF86C1B0860DFF8680B40788DF843
:100460000100DFF8600B00788DF80000CAE6DFF8C5
:10047000540BC0788DF80100DFF8480B80788DF8B8
:100480000000BFE6DFF83C0B40798DF80100DFF893
:10049000340B00798DF80000B4E6DFF8280BC07942
:1004A0008DF80100DFF81C0B80798DF80000A9E6BB
:1004B000DFF8100B407A8DF80100DFF8080B007AA6
:1004C0008DF800009EE6DFF8FC0AC07A8DF8010086
:1004D000DFF8F00A807A8DF8000093E6DFF8E00A92
:1004E00000684FF6F7710840DFF8D41A08600C2155
:1004F000DFF8D40A01F0E4F9DFF8C40A006850F02C
:100500000C00DFF8BC1A0860DFF8BC0A40788DF8F0
:100510000100DFF8B40A00788DF8000072E6DFF819
:10052000A80AC0788DF80100DFF89C0A80788DF861
:10053000000067E6DFF8900A40798DF80100DFF8E7
:10054000880A00798DF800005CE6DFF87C0AC07943
:100550008DF80100DFF8700A80798DF8000051E60F
:10056000DFF8640A407A8DF80100DFF85C0A007A4F
:100570008DF8000046E6DFF8500AC07A8DF80100D9
:10058000DFF8440A807A8DF800003BE6BDF80200EF
:10059000ADF8000036E6BDF804005FEA400818EB4D
:1005A0000500C11C89B2DFF8EC0901F0DCF9ADF8F7
:1005B0000400DFF8E009ADB21FFA88F818EB050176
:1005C00008449DF80410C170DFF8C809ADB21FFAE5
:1005D00088F818EB050108449DF80510017101F039
:1005E00063B85BF08000DFF8AC19ADB22944487005
:1005F000BDF80400802803DABDF80400002806D105
:100600000320DFF89019ADB22944887005E002207C
:10061000DFF88019ADB229448870E91C89B2DFF88F
:10062000740901F0A0F9ADF804009DF80400DFF8AA
:100630006419ADB22944C8709DF80500DFF854195B
:10064000ADB2294408716E1D01F02EB89AF8000071
:10065000002801F0318000200090ADB20AEB0500C7
:1006600080788DF80100ADB20AEB0500C0788DF8F6
:100670000000ADB20AEB050000798DF80500ADB2BF
:100680000AEB050040798DF804009AF80000DFF8C5
:1006900004190870ADB2002D09D09AF80100DFF8F6
:1006A000F41848709AF80200DFF8E81888700226FB
:1006B0000098B0F58060FF2805D90098B0F570600B
:1006C000802880F01A82009F4FF481603F1A27D063
:1006D0007F1E4CD07F1E4CD07F1E7DD07F1E00F031
:1006E00099807F1E00F0B9807F1E00F0D9807F1EA8
:1006F00000F0F9807F1E00F019817F1E00F0348128
:100700007F1E00F04F817F1E00F06F817F1E00F082
:100710008F817F1E00F0AF817F1E00F0CF81EBE163
:100720009DF804209DF80510002001F025F89DF8A3
:100730000500DFF88018087000BF9DF804209DF8C0
:100740000510012001F018F89DF80500DFF8681881
:10075000087000BF00220021112001F00DF800BF39
:1007600000220021102001F007F80026C5E1002634
:10077000C3E1BDF8040010F4C0795FEAC9501ED48B
:100780000022FF21002000F0F7FFFF20DFF82418EF
:10079000087000BF0022FF21012000F0EDFFFF20C4
:1007A000DFF81418087000BF00220021102000F0AC
:1007B000E3FF00BF00220021112000F0DDFFDFF881
:1007C000FC07006810F4CC6050EA0909DFF8EC0778
:1007D000C0F80090002690E19DF80500DFF8E417CE
:1007E0004870DFF8DC0700684FF6FB710840DFF85F
:1007F000D017086001220121DFF8380E01F04EF811
:10080000DFF8BC07006850F00C00DFF8B417086090
:10081000002672E19DF80400DFF8A81788709DF8A3
:100820000500DFF8A017C870DFF8940700684FF6DE
:10083000FB710840DFF88817086002220221DFF808
:10084000F80D01F02BF8DFF87807006850F00C0085
:10085000DFF86C17086000264FE19DF80400DFF810
:10086000641708719DF80500DFF858174871DFF824
:10087000500700684FF6FB710840DFF84417086026
:1008800004220221DFF8340E01F008F8DFF8300707
:10089000006850F00C00DFF82817086000262CE1F3
:1008A0009DF80400DFF81C1788719DF80500DFF83B
:1008B0001417C871DFF8080700684FF6FB7108408D
:1008C000DFF8FC16086006220221DFF8F40D00F0C4
:1008D000E5FFDFF8EC06006850F00C00DFF8E016EA
:1008E0000860002609E19DF80400DFF8D8160872B8
:1008F0009DF80500DFF8CC164872DFF8C4060068E2
:100900004FF6FB710840DFF8B81608600822022194
:10091000DFF8B00D00F0C2FFDFF8A406006850F069
:100920000C00DFF89C1608600026E6E09DF8040045
:10093000DFF890168872DFF8880600684FF6FB71C2
:100940000840DFF87C1608600A220121DFF87C0DE0
:1009500000F0A4FFDFF86806006850F00C00DFF834
:10096000601608600026C8E09DF80500DFF85816FC
:100970004870DFF84C0600684FF6F7710840DFF862
:100980004016086001220121DFF8440D00F086FFC7
:10099000DFF82C06006850F00C00DFF82416086021
:1009A0000026AAE09DF80400DFF81C1688709DF868
:1009B0000500DFF81416C870DFF8040600684FF66B
:1009C000F7710840DFF8F815086002220221DFF80D
:1009D000040D00F063FFDFF8E805006850F00C003C
:1009E000DFF8DC150860002687E09DF80400DFF8DA
:1009F000D81508719DF80500DFF8CC154871DFF8AF
:100A0000C00500684FF6F7710840DFF8B4150860BC
:100A100004220221DFF8C00C00F040FFDFF8A0053F
:100A2000006850F00C00DFF898150860002664E0BC
:100A30009DF80400DFF8901588719DF80500DFF837
:100A40008815C871DFF8780500684FF6F77108401F
:100A5000DFF86C15086006220221DFF8800C00F038
:100A60001DFFDFF85C05006850F00C00DFF8501542
:100A70000860002641E09DF80400DFF84C1508727C
:100A80009DF80500DFF840154872DFF8340500686E
:100A90004FF6F7710840DFF8281508600822022198
:100AA000DFF83C0C00F0FAFEDFF81405006850F0A7
:100AB0000C00DFF80C15086000261EE09DF804000D
:100AC000DFF804158872DFF8F80400684FF6F77154
:100AD0000840DFF8EC1408600A220121DFF8040C5A
:100AE00000F0DCFEDFF8D804006850F00C00DFF8FE
:100AF000D0140860002600E00226F6B2002E23D0B3
:100B00005BF08000DFF88C14ADB229444870DFF848
:100B10008404ADB228448670E91C89B2DFF87404FD
:100B200000F021FFADF804009DF80400DFF8641424
:100B3000ADB22944C8709DF80500DFF85814ADB275
:100B4000294408716E1D2FE05FF001080FE01FFAC5
:100B500088F80AEB0800ADB2405DDFF838141FFAE0
:100B600088F8ADB215EB0802885418F101081FFA95
:100B700088F8B8F1060FEADBA91D89B2DFF8140482
:100B800000F0F1FEADF804009DF80400DFF8041455
:100B9000ADB2294488719DF80500DFF8F813ADB2B5
:100BA0002944C87115F1080600F07EBD9AF80000CE
:100BB000002800F0818500200090ADB20AEB05000E
:100BC00080788DF80100ADB20AEB0500C0788DF891
:100BD0000000ADB20AEB050000798DF80500ADB25A
:100BE0000AEB050040798DF804009AF80000DFF860
:100BF000A4130870ADB2002D09D09AF80100DFF8F7
:100C0000941348709AF80200DFF88813887002265F
:100C10000098B0F58060B0F5386F80F00082BDF8C4
:100C20000400002800F0FB81BDF80400802880F259
:100C3000F6810098BDF804100818B0F5786F00F23E
:100C4000EE8100265FF0000801E018F1010840463F
:100C5000BDF8041080B2884280F0E18100984FF422
:100C60008161401A28D0401E6ED0401E6DD0401EBB
:100C700000F0AF80401E00F0B780401E00F0C98039
:100C8000401E00F0DB80401E00F0ED80401E00F0B2
:100C9000FF80401E00F01E81401E00F02681401E95
:100CA00000F03881401E00F04A81401E00F05C8157
:100CB000401E00F08B81ABE1ADB20AEB05001FFADC
:100CC00088F800EB4800027AADB20AEB05001FFA83
:100CD00088F800EB4800C179002000F04DFDADB26E
:100CE0000AEB05001FFA88F800EB4800C079B1490B
:100CF000087000BFADB20AEB05001FFA88F800EBE0
:100D00004800027AADB20AEB05001FFA88F800EB42
:100D10004800C179012000F02FFDADB20AEB0500BB
:100D20001FFA88F800EB4800C079A349087000BF9B
:100D300000220021112000F01FFD00BF0022002131
:100D4000102000F019FD63E162E1ADB20AEB05008D
:100D50001FFA88F800EB4800C0798DF80900ADB2A1
:100D60000AEB05001FFA88F800EB4800007A8DF8BE
:100D70000800029810F4C0700290BDF80800C00589
:100D80001CD40022FF21002000F0F6FCFF2089493E
:100D9000087000BF0022FF21012000F0EDFCFF20C1
:100DA0008549087000BF00220021102000F0E4FCFB
:100DB00000BF00220021112000F0DEFC02987F49D4
:100DC000096811F4CC610843029002987B490860DD
:100DD0001EE1ADB20AEB05001FFA88F800EB4800EF
:100DE000C0797849487013E1ADB20AEB05001FFAEB
:100DF00088F800EB4800007A72498870ADB20AEBBF
:100E000005001FFA88F800EB4800C0796D49C870EA
:100E1000FEE0ADB20AEB05001FFA88F800EB4800CF
:100E2000007A68490871ADB20AEB05001FFA88F82C
:100E300000EB4800C07963494871E9E0ADB20AEBC4
:100E400005001FFA88F800EB4800007A5D498871B8
:100E5000ADB20AEB05001FFA88F800EB4800C07934
:100E60005849C871D4E0ADB20AEB05001FFA88F802
:100E700000EB4800007A53490872ADB20AEB050056
:100E80001FFA88F800EB4800C0794E494872BFE06D
:100E9000ADB20AEB05001FFA88F800EB4800007AB3
:100EA00048498872464800684FF6FB71084044493B
:100EB000086001220A21DFF87C0700F0EFFC4048BF
:100EC000006850F00C003E490860A1E020000020BE
:100ED00000020020ADB20AEB05001FFA88F800EB13
:100EE0004800C0793849487092E0ADB20AEB05007D
:100EF0001FFA88F800EB4800007A33498870ADB2D9
:100F00000AEB05001FFA88F800EB4800C0792E496B
:100F1000C8707DE0ADB20AEB05001FFA88F800EB5F
:100F20004800007A28490871ADB20AEB05001FFAA3
:100F300088F800EB4800C0792349487168E0ADB2F9
:100F40000AEB05001FFA88F800EB4800007A1E49FA
:100F50008871ADB20AEB05001FFA88F800EB480073
:100F6000C0791949C87153E0ADB20AEB05001FFA08
:100F700088F800EB4800007A13490872ADB20AEB1A
:100F800005001FFA88F800EB4800C0790E49487246
:100F90003EE000BF000800208801002090010020F2
:100FA00098010020A0010020A8010020B00100202D
:100FB000B80100201D0000201E00002000000B4092
:100FC00000800C40000000200C000020ADB20AEBB5
:100FD00005001FFA88F800EB4800007ADFF80817D0
:100FE0008872DFF8080700684FF6F7710840DFF8ED
:100FF000FC16086001220A21DFF8D40600F04EFC3E
:10100000DFF8E806006850F00C00DFF8E016086032
:101010000098401C0090F6B2002E3FF416AEF6B2D7
:10102000002E2FD05BF08000DFF8C416ADB229444B
:101030004870BDF80400812806DB0320DFF8B016F5
:10104000ADB22944887005E00220DFF8A416ADB2E5
:1010500029448870E91C89B2DFF8940600F083FC0B
:10106000ADF804009DF80400DFF88416ADB2294401
:10107000C8709DF80500DFF87816ADB229440871F4
:101080006E1D2FE05FF001080FE01FFA88F80AEBF1
:101090000800ADB2405DDFF858161FFA88F8ADB20F
:1010A00015EB0802885418F101081FFA88F8B8F106
:1010B000060FEADBA91D89B2DFF8340600F053FC05
:1010C000ADF804009DF80400DFF82416ADB2294401
:1010D00088719DF80500DFF81816ADB22944C87173
:1010E00015F10806E0E29AF80000002800F0E4821A
:1010F0008E1C5FF000080BE01FFA88F81AF8080051
:10110000DFF8EC151FFA88F801F8080018F101085B
:101110004046310080B289B28842EDD3C4E29AF8E9
:101120000000002800F0C88215F109069AF80000B6
:10113000DFF8BC150870ADB2002D09D09AF8010097
:10114000DFF8AC1548709AF80200DFF8A415887033
:101150001120DFF89C15ADB2294448700420DFF857
:101160009015ADB2294488704820DFF88415ADB2DF
:101170002944C8700120DFF87815ADB22944087100
:101180000120DFF86C15ADB2294448710520DFF865
:101190006015ADB229448871E91D89B2DFF85005A8
:1011A00000F0E1FBADF804009DF80400DFF8401505
:1011B000ADB22944C8719DF80500DFF83415ADB211
:1011C0002944087270E29AF80010002900F0748235
:1011D0009AF80010DFF818251170ADB2002D09D073
:1011E0009AF80110DFF8082551709AF80210DFF81C
:1011F00000259170ADB20AEB050189780E2940F007
:10120000E5812B21DFF8E824ADB22A4451700E218C
:10121000DFF8DC24ADB22A449170ADB20AEB0501CF
:10122000C978012940F08C800120DFF8C414ADB2E8
:101230002944C8700120DFF8B814ADB22944087100
:101240000020DFF8AC14ADB2294448710020DFF86B
:10125000A014ADB2294488710320DFF89414ADB214
:101260002944C8710020DFF88814ADB229440872FF
:1012700015F10A08DFF87C14DFF874041FFA88F807
:101280004044FEF71DFFDFF86814ADB229444872F0
:10129000C0B210EB08080120DFF854141FFA88F8D8
:1012A00001F8080018F10108DFF84C14DFF84004D9
:1012B0001FFA88F84044401CFEF702FFDFF83014A4
:1012C0001FFA88F801F80800C0B2401C10EB0808AB
:1012D0000220DFF81C141FFA88F801F8080018F142
:1012E0000108DFF81814DFF808041FFA88F84044F2
:1012F000401CFEF7E5FEDFF8F8131FFA88F801F846
:101300000800C0B2401C10EB0808414689B2DFF863
:10131000E00300F028FBADF804009DF80400DFF8BE
:10132000D0131FFA88F801F808009DF80500DFF8CF
:10133000C0131FFA88F84144487018F10206B3E15F
:10134000ADB20AEB0501C978022940F0A280022063
:10135000DFF89C13ADB22944C8700220DFF8901367
:10136000ADB2294408710020DFF88413ADB22944DE
:1013700048710020DFF87813ADB229448871042049
:10138000DFF86C13ADB22944C8710320DFF8601395
:10139000ADB22944087215F10A08DFF86413D44885
:1013A0001FFA88F84044FEF78BFED149ADB22944BC
:1013B0004872C0B210EB08080420CD491FFA88F823
:1013C00001F8080018F10108CE49C9481FFA88F849
:1013D0004044401CFEF774FEC5491FFA88F801F826
:1013E0000800C0B2401C10EB08080520C0491FFAD5
:1013F00088F801F8080018F10108C349BC481FFA31
:1014000088F84044401CFEF75BFEB9491FFA88F893
:1014100001F80800C0B2401C10EB08080620B449CF
:101420001FFA88F801F8080018F101085FF00109B7
:101430004A46A5A1AE481FFA88F84044401C00F077
:10144000D1FBAB481FFA88F84044401C00F0E4FB95
:10145000A7491FFA88F801F80800C0B2401C10EB39
:101460000808414689B2A24800F07DFAADF80400B0
:101470009DF804009E491FFA88F801F808009DF8BD
:1014800005009B491FFA88F84144487018F102068C
:101490000AE1ADB20AEB0501C978042940F0968053
:1014A000ADB20AEB05010979072980F28F8004218A
:1014B0008F4AADB22A44D17084218D4AADB22A44FC
:1014C000117100218A4AADB22A4451710021884A23
:1014D000ADB22A4491710121854AADB22A44D1713D
:1014E000ADB20AEB05010979814AADB22A44117205
:1014F000ADB20AEB05010979002906D17D497C4886
:10150000ADB228440A30FEF7DBFDADB20AEB0501AF
:101510000979012906D178497548ADB228440A30C5
:10152000FEF7CEFDADB20AEB05010979022906D11D
:1015300072496F48ADB228440A30FEF7C1FDADB222
:101540000AEB05010979032906D16D496848ADB256
:1015500028440A30FEF7B4FDADB20AEB0501097963
:10156000042906D167496248ADB228440A30FEF723
:10157000A7FDADB20AEB05010979052906D162493B
:101580005B48ADB228440A30FEF79AFD5849ADB227
:1015900029444872C0B2401910F10A08414689B284
:1015A000534800F0E0F9ADF804009DF804005049FC
:1015B0001FFA88F801F808009DF805004C491FFA49
:1015C00088F84144487018F102066DE0ADB20AEBAC
:1015D0000500407850F080004549ADB2294448707C
:1015E00002204349ADB229448870E91C89B24048C1
:1015F00000F0B9F9ADF804009DF804003C49ADB223
:101600002944C8709DF805003949ADB229440871D4
:101610006E1D49E09AF8000000284DD045F2555063
:101620003A49086000203A4908604CF6CC403749F6
:101630000860FEE701000020020000209AF8000088
:10164000002839D06E1D9AF8000029490870ADB203
:10165000002D07D09AF80100254948709AF8020039
:1016600023498870ADB20AEB0500407850F0800045
:101670001F49ADB22944487001201D49ADB229442B
:101680008870E91C89B21A4800F06DF9ADF80400C1
:101690009DF804001649ADB22944C8709DF80500B4
:1016A0001349ADB229440871A4B2012C04D1B6B2D9
:1016B00031000F4800F0B4F9BDE8F78F04000020B6
:1016C0000600002008000020256C75000A0000209C
:1016D0000D0000200E00002010000020120000204D
:1016E00014000020160000200C00002000800C4098
:1016F0000008002088470008904700083447000889
:101700002A2A0008A04700089847000800800640E1
:101710000480064072B600211BE05F4A12684FF653
:10172000F7731A405C4B1A6000BF00BF00BF00BFD8
:1017300000BF00BF4000584A12684FF6FB731A40C2
:10174000554B1A6000BF00BF00BF00BF00BF00BF05
:10175000491C08290ED2504A126852F004024E4B1E
:101760001A600206D9D54C4A126852F008024A4B58
:101770001A60D9E762B6704738B50C0015004649C3
:1017800009684FF6FB721140434A116042490968EB
:101790004FF6F9721140404A116000BFC0B2FFF726
:1017A000B9FF2000C0B2FFF7B5FF2800C0B2FFF7B5
:1017B000B1FF00BF3848006850F0020036490860A9
:1017C00031BD0000002072B6334909684FF6BF7280
:1017D0001140314A1160002119E010F0FE002E4A3C
:1017E000126852F020022C4B1A6000BF00BF00BFED
:1017F00000BF00BF00BF00BF00BF00BF00BF264A40
:1018000012684FF6DF731A40234B1A60491CC9B2A5
:1018100008290CDA00BF00BF00BF00BF00BF4000B6
:101820001D4A1268D206D8D550F00100D7E762B63B
:10183000C0B2704772B6002120E0174A12684FF616
:10184000BF731A40144B1A6000BF00BF00BF4000B6
:10185000114A126852F020020F4B1A6000BF00BFFD
:1018600000BF00BF00BF00BF00BF00BF0A4A126830
:101870004FF6DF731A40084B1A60491CC9B2082999
:1018800008DA0206D9D5044A126852F04002024B27
:101890001A60D9E762B6704700800A4038B5040084
:1018A0000D00500010F0F700FFF7C4FF04E02078AF
:1018B000FFF7C0FF641C6D1EADB2002DF7D131BD26
:1018C00038B504000D000120FFF7B4FF04E0FFF776
:1018D00079FF2070641C6D1EADB2002DF7D131BDB3
:1018E00000BF40F2013096490860682095490860C1
:1018F0000B2095490860782094490860002094499D
:10190000086040F2FF709349086010209249086017
:101910000020924908608020914908608020914908
:101920000860704740F201208F49086068208F49A5
:1019300008600B208E49086070208E4908600020E6
:101940008D49086040F2FF708C49086010208C4976
:10195000086000208B4908604020814908604020D1
:1019600080490860704718B44FF6FF72ADF8002048
:101970009DF8002003785A40401C9DF80130824CAD
:10198000D2B2A45C63408DF80030804BD2B29A5C36
:101990008DF80120491E89B20029E9D1BDF8000067
:1019A00012BC70477A48006800BF7A49096860290C
:1019B00008D27949774A1268885476480088401CD2
:1019C0007449088075480068C006EBD50520744945
:1019D00008607448006830F002007249086070477F
:1019E0007148006800BF71490968B1F5847F08D269
:1019F0006F496E4A126888546C480088401C6B49D5
:101A000008806C480068C006EAD505206A4908606D
:101A10006448006830F004006249086070470000C4
:101A200010B4002932D0B1F5847F01D94FF484710C
:101A3000624A92F8282012F00F0FF9D15F4A127A09
:101A400012F00F0FF4D104225D4B1A6001225D4B9E
:101A50001A60002203E0835C5B4CA354521C8A4250
:101A6000F9DBBFF34F8F491E57480818534A1062DD
:101A7000564850EA011051498862042054490860D0
:101A800004205449086002203449086010BC7047A3
:101A900010B4002952D0B1F5847F01D94FF484717C
:101AA0004D4A4E4B1A604FF400624D4B1A6040F2A3
:101AB00001122D4B1A60414A127A12F00F0FFAD11F
:101AC0003E4A92F8282012F00F0FF4D101223C4B2D
:101AD0001A6001223B4B1A60002203E0835C3A4CFF
:101AE000A354521C8A42F9DBBFF34F8F491E36487C
:101AF0000818324A1060354850EA01102F498860B2
:101B000001203349086001203249086002201D4944
:101B100008602A48007A10F00F0FFAD11F480068B9
:101B20000007FBD45FF4A8202C4908604FF4005054
:101B30002B49086040F201200B49086010BC704737
:101B40003080034024800340288003402C800340E1
:101B50003480034044800340388003404880034081
:101B600080E200E000E100E0300003402400034098
:101B7000280003402C00034034000340440003408D
:101B8000380003404800034044440008444500082E
:101B900000000340FC010020280100201800034041
:101BA000C401002018000020008003400002002033
:101BB0002000002018800340C801002000040020FD
:101BC0002C8002404C800240080900200100B4C073
:101BD00024800240288002400044050018000B4089
:101BE00008000B400CB41CB5044604A801900A463A
:101BF000009401AB694607487844183000F02CF88F
:101C0000009A0021117000285CBF0098001B16BCD0
:101C10005DF80CFB3B00000000F10103810704D0DC
:101C200010F8011B89B18107FAD10268B2F10131C4
:101C3000914311F0803F04BF50F8042FF6E710F8ED
:101C4000011B11B110F8011BFBE7C01A70470268B5
:101C5000531C0360117070472DE9F04FA1B082460C
:101C600001AE002017461D467160B0620DF14409B7
:101C70000AE017F8011B7068D0470028706000F078
:101C8000B982B06A401CB0623878010001D1B06AF4
:101C9000B2E22528EDD1002030617061B061F061C1
:101CA0003062706201E040F0010017F8011F202946
:101CB000F9D023290DD02B2904D02D2906D0302985
:101CC0000AD00CE040F0020080B2EEE740F00400E1
:101CD000FAE740F00800F7E740F01000F4E72A299F
:101CE0000ED12968296051F8042B2960002A32633B
:101CF00004D5514240F00400316380B27F1C13E0F0
:101D0000002131630BE0316B6FF00043994205D045
:101D100001EB810302EB4301303931637F1C3A78D8
:101D2000A2F130010A29EED339782E2903D04FF0E1
:101D3000FF31F1621FE017F8011F2A2907D1296836
:101D400029607F1C51F8042B2960F26213E0002106
:101D5000F1620BE0F16A6FF00043994205D001EBAC
:101D6000810302EB43013039F1627F1C3A78A2F122
:101D700030010A29EED3B0860FF69440397800F08E
:101D800055FE08B117F8010B8DF83A009DF83A009E
:101D9000682802BF39786829622005D06C2804BF02
:101DA00038786C2803D171208DF83A007F1C11A877
:101DB000F06017F8014BB4F125002AD01C3800F070
:101DC000CA80001F022840F2C680133800F0EA8063
:101DD000093800F0C080801E00F05481401E00F0E1
:101DE0002B81401E022840F2B680001F00F02481A3
:101DF000401F00F08180401E00F0D480401E26D09D
:101E0000C01E0BD0801E00F0CD80C01E00F0CA8026
:101E100042E125208DF84400012046E12868286031
:101E200050F8048B2860C6F80880F46A002C04D5AA
:101E30004046FFF7F1FE044607E0224600214046F7
:101E400000F000FE08B1A0EB080474612EE12968DF
:101E50002960002251F8040B29604FF03C0E00214C
:101E6000CDE9000111A8B060DDE900019142F468FC
:101E700008BF904201D1F26AC2B100F00F033033C3
:101E8000DBB23A2BA8BF2733AEF101020009A354FD
:101E9000964640EA017009090022914208BF90422B
:101EA00004D0B26804EB0E039A42E6D304EB0E01B1
:101EB000B160CEF13C00F16A7061884207DA081A1D
:101EC000F0614FF6EF71B08E0840B086EEE0002969
:101ED00040F1EC8096F8341001F01401102940F024
:101EE000E580316B3269891AF269891A081A01286A
:101EF000C0F2DC80F061D9E09DF83A0062281AD087
:101F0000682806D06A280CD06C281CD0712808D00C
:101F100019E02868286050F8041B2860B06A08801F
:101F2000C4E02868286050F8042B2860B06AC11704
:101F3000C2E90001BAE02868286050F8041B286054
:101F4000B06A0870B2E02868286050F8041B286066
:101F5000B06A0860AAE02868C01D20F007022A6065
:101F6000D2E9000108322A60CDE90001002902D53A
:101F700030692D2109E0B08E810702D530692B210F
:101F800003E0C00705D53069202109F80010401C86
:101F9000306111A831690844B0602146684600F0FC
:101FA000EBF983E09DF83A006C280DD0712818BF3A
:101FB0006A2809D12868C01D20F007022A60D2E9EA
:101FC000000108322A6005E02968296051F8040BF5
:101FD00029600021CDE900019DF83A00682803D16D
:101FE000DDE9000180B20BE0622803D1DDE90001E8
:101FF000C0B205E0742818BF7A2804D1DDE90001D9
:102000000021CDE9000196F83400000731D5DDE963
:1020100000230020834208BF82422AD044F02000DF
:10202000782826D13069302109F80010401C411C65
:10203000316109F800401CE09DF83A00294600F0A3
:10204000DEF8CDE90001DDE9002300218B4202DA50
:1020500030692D2109E0B08E810702D530692B212E
:1020600003E0C00705D53069202109F80010401CA5
:10207000306111A831690844B0602146684600F01B
:10208000F5F813E0012030612868286050F8041B3F
:1020900028608DF8441009E025208DF844000120C7
:1020A00030611CB189F8014002203061306B316928
:1020B000401AF169401A7169401A316A401AB169CF
:1020C000401A716AA0EB010896F83400400711D459
:1020D0002020B8F1010F8DF840000BDB44460123AE
:1020E00010AA6946504600F07CFC002840F082802F
:1020F000641EF4D1D6F810B0BBF1000F11AC0CD0B7
:1021000014F8011B7068D0470028706072D0B06A64
:10211000401CBBF1010BB062F2D130208DF84000C1
:10212000F469012C09DB012310AA6946504600F02E
:1021300058FC00285ED1641EF5D1D6F814B0B468FE
:10214000BBF1000F0CD014F8011B7068D0470028B9
:1021500070604FD0B06A401CBBF1010BB062F2D18D
:1021600030208DF84000346A012C09DB012310AACD
:102170006946504600F035FC00283BD1641EF5D17D
:10218000B0687169D6F818B04418BBF1000F0BD0D5
:1021900014F8011B7068D047706058B3B06A401CD7
:1021A000BBF1010BB062F3D130208DF84000746AAE
:1021B000012C08DB012310AA6946504600F011FCEF
:1021C000C0B9641EF6D196F8340040077FF55CADC7
:1021D0002020B8F1010F8DF84000FFF655AD012326
:1021E00010AA6946504600F0FCFB18B9B8F1010886
:1021F000F5D149E54FF0FF3021B0BDE8F08F6228FE
:1022000026D068281DD06A2808D06C2827D07128CD
:1022100004D0742823D07A280CD020E00868C01D90
:1022200020F007000860D0E9002308300860194654
:10223000104670470A680A6052F8040B0A600021D1
:1022400070470A680A6052F8040B0A6000B20BE09B
:102250000A680A6052F8040B0A6040B204E00A6897
:102260000A6052F8040B0A60C11770472DE9F34366
:10227000054608462F696F2808BF082405D041F09D
:102280002001782914BF0A2410243C26D5E9002314
:10229000642818BF69289046994606D100218B42D0
:1022A00003DAD8F1000869EB49090020814508BF2D
:1022B00080450CD1286B50B9082C38D195F83800DE
:1022C000000734D530203B2687F83B002FE0701EF6
:1022D00000900646404649462246E31700F0DEFBE2
:1022E00002F13000C0B23A2803DB9DF804105139E6
:1022F0000818B855494640462246E31700F0CEFB81
:10230000804689460020814508BF804503D0E868A3
:10231000B9198842DBD3082C09D195F83800000799
:1023200005D5B85D302802D0761E3020B855B919D1
:10233000E960C6F13C00296BA861884208DA081AF6
:1023400028624FF6EF71288F08402887BDE8F38395
:1023500000290ED595F8381001F01401102908D184
:10236000696B6A69891A2A6A891A0E1A012EA8BF2E
:102370002E62BDE8F38300002DE9F24F04468EB0D3
:10238000D4E90001CDE9020104AF9DF8380040F026
:10239000200BBBF1610F0AD0206B002848BF06203C
:1023A00004D408BFBBF1670F01D10120206361682D
:1023B000C1F30A5040F2FF7290421CD1080304BFDF
:1023C0002068002809D10320A0619DF838006138F9
:1023D0001A2835D30FF24C6108E00320A0619DF864
:1023E000380061381A2828D30FF23061E0680322E0
:1023F00000F0CCFBBDE1012815DA204600F001FC1D
:10240000012810DB00250020BBF1610F1FD1E1681E
:1024100030220A708A1CE2609DF83820612A0CBFC5
:10242000782258220FE0626840F2FE3161F31E52BA
:10243000451A62604FF0FF30E6E70FF2DC51D5E756
:102440000FF2DC51D2E74A706169891C616110B9F1
:102450000026002584E1BBF1610F40F09880206BDD
:10246000D4E900AB00284CBF2126461CDDE902015F
:102470000022002300F0E8FB36B23ABF8BF00040A8
:10248000CDE902A0CDE902AB06F101082D1FB8F19C
:10249000010F8DF810200DF1110736DBDDE9020187
:1024A0000022002300F0E8FB2FD21C2102A800F03C
:1024B000FBFBDDE9020100F07DFCA8F10708B8F1A3
:1024C000010F814609DB00F0A1FC02460B46DDE965
:1024D000020100F0B3FCCDE90201F81D072105E07F
:1024E00009F00F0200F8012D4FEA2919B9F1010F87
:1024F00001DB491EF4D5491E5CBF002200F8012D06
:10250000F9D5C71DB8F1010FC8DA0DF11100391A5C
:10251000B142B8BF0E4636B230000DF111072FD4CC
:10252000884206DA04A9014449780829A8BF0F2186
:1025300000DA002104AA024400E0761E12F80139F4
:10254000401E8B42F9D00F2904D104A901444A78D6
:10255000521C4A70002802D504AF761C2D1D36B2DD
:10256000701E0DD439180A783032D2B23A2A03DB01
:102570009DF838303A3B9A18401E01F80129F2D5EF
:10258000206B002840F1EC80701E2063E8E0DDE95C
:1025900002010022002300F057FB3CBF81F0004104
:1025A000CDE902012DB247F2975068434B49DFF85D
:1025B000309190FBF1F52DB2C5F1070ABAF1010F88
:1025C00090461CDBDDE902675FEACA7007D5424628
:1025D0004B463046394600F0F1FC06460F46404671
:1025E000494642464B464FEA6A0A00F0E7FCBAF118
:1025F000000F80468946E7D1CDE9026724E0CAF1A1
:10260000000A0026374F14E05FEACA7007D5424639
:102610004B463046394600F0D1FC06460F46404650
:10262000494642464B4600F0C9FC4FEA6A0A8046DA
:102630008946BAF1000FE7D1DDE9020132463B4697
:1026400000F08EFDCDE90201BBF1660F216BDFF8D2
:1026500098900CBF05F10A0006204618142EA8BF5A
:10266000132630208DF810000DF11107012E3DDBEF
:10267000DDE9020100F0B4FB07F1080104220A239E
:10268000B0FBF3F303EB8307A0EB4700303001F816
:10269000010C0A20B3FBF0F000EB8007A3EB47032B
:1026A0003033521E01F8023DE9D1083E012E01F1FE
:1026B0000807DBDBDDE9020100F092FB00F0B0FB74
:1026C00002460B46DDE9020100F0B8FB00224B4652
:1026D00000F074FCCDE90201CAE700BFA08601004A
:1026E000000024400000F03F84D797410DF1110015
:1026F000381A0DF1110702E0401E6D1E7F1C39785B
:102700003029F9D0BBF1660F08BF691C04D0BBF1BA
:10271000650F0CBF01210021226B8E1836B2B0422A
:10272000B8BF064636B231001AD4814204DA785C6A
:102730003528A8BF392000DA30207A18521E00E070
:10274000761E12F80139491E8342F9D0392802D188
:10275000785C401C7854002902D57F1E761C6D1CC5
:102760002DB29DF83810009533B23A46204600F05D
:1027700003F80FB0BDE8F08F2DE9F043054685B0B2
:102780001F46D5F83080012F8946164602DA012708
:102790000FF2942649F02000BDF93040662808BFAA
:1027A000641C17D0672840F0848014F1040FC0F235
:1027B0008680444580F2838095F83800641C0007C9
:1027C00002D44745B8BFB84624B2B8EB040848BFA6
:1027D0004FF0000824B2E868A969012C27DA4A1CE6
:1027E00030234354B8F1010F03DA95F8380000079D
:1027F00003D5E9682E208854521C18EB040FB8BF8B
:10280000C8F1000424B260426862A044B845AA61DD
:10281000B8BF4746E868AB693FB2EF613A46314618
:10282000184400F0B3F9A8EB0700A862C2E0224602
:102830009742084418DA3A46314600F0A7F9A969E8
:102840007918E01BB8F1010FA961686203DA95F805
:102850003800000705D5EA682E205054E869401C6E
:10286000E861C5F82880A5E0314600F08FF9A86935
:1028700020183F1BB8F1010F03DA95F8381009074B
:1028800003D5EA682E211154401CA8613FB2B84517
:10289000B8BF4746E868AB693FB23A4631191844B9
:1028A00000F074F9A8693818A861A8EB07006862FD
:1028B00080E0B9F1610F16D14FF0700918E047457B
:1028C00004DA95F83810090758BFB846B8F101087E
:1028D00048BF4FF00008B9F1670F14BF4FF045092A
:1028E0004FF0650904E0B9F1410F08BF4FF05009FE
:1028F000A969EB68481CA861B8F1010F16F8012B13
:102900005A5403DA95F83810090719D5EA68431CB8
:10291000AB612E211154B8F1010F11DB7F1E3FB2C4
:10292000B845B8BF4746E8683FB23A463146184412
:1029300000F02CF9A8693818A861A8EB07006862B4
:10294000E868A9690144200081F8009003D42B2095
:1029500048708E1C03E02D224A708E1C64420027B2
:102960000DF1080808E00A22684600F024FD0198ED
:1029700008F8010B7F1C009C21B20129F3DA022F19
:1029800006DA49F02000652804BF302006F8010B64
:102990004FB9302006F8010B07E07F1E02A8C05D8A
:1029A000303006F8010B012FF7DAE868A96908440E
:1029B000301AE86195F8380000F0140010280DD1A5
:1029C0006869A9690818696A0818E9690818A96A8C
:1029D0000818696B8842BCBF081A286205B0BDE8B8
:1029E000F083F8B504460D4616461F46002077B121
:1029F00016F8011BA868A047A86030B1E86A401C1F
:102A0000E86200207F1EF3D1F2BD4FF0FF30F2BD2F
:102A1000686A6C747A4C00006E616E004E414E0024
:102A2000696E6600494E4600300041000278C9B226
:102A30008A421AB11CBF10F8012FF9E718BF002015
:102A40007047FEE7C9B2830706D0521E22D310F8A2
:102A5000013B9942F7D11FE0083A13D302F1040277
:102A600041EA012141EA014150F8043B121F21BF14
:102A70004B40A3F1013C2CEA030C1CF0803FF3D047
:102A8000C9B2001F083210F8013B521E28BF91EA5C
:102A9000030FF8D818BF0120401E70471B4213D106
:102AA000094236D12AB18446B0FBF2F002FB10C2D3
:102AB000704700F087BCFCD30022002370470B0056
:102AC0000200002100207047904271EB030CF6D306
:102AD00070B5B1FA81F4B3FA83F52C1BA340C4F1AD
:102AE000200532FA05F63343A2405FF00046E64087
:102AF00002E05B085FEA3202841A71EB030524BF2F
:102B0000204629467641F4D302000B003000002114
:102B100070BD012ACFD970B5140C20D0B1FA81F460
:102B2000B2FA82F5C4F120046419B4F12006D6D3B8
:102B3000B2405FF00044F440002502E052085FEA32
:102B40003303C61A71EB020E24BF3046714664414E
:102B50006D41F3D302000B002000290070BD0C462C
:102B6000B1FBF2F102FB11452D0445EA1045B5FB1E
:102B7000F2F402FB145580B240EA0545B5FBF2F0D1
:102B800002FB105240EA044070BDFEE762B38B07BF
:102B900008D0521E11F8013B00F8013B00F02480E0
:102BA0008B07F6D1830740F0208000BF103A07D38F
:102BB00030B4B1E83810103AA0E83810F9D230BC7F
:102BC000530724BFB1E80810A0E8081044BF51F82B
:102BD000043B40F8043BD20724BF31F8022B20F815
:102BE000022B44BF0B7803707047083A07D3B1E853
:102BF0000810083A40F8043B40F804CBF7D25307DA
:102C0000E4E730B4436803F000420121C3F3130347
:102C10004360002B04BF0368002B08D10DE003685C
:102C2000DD0F45EA440444605B000360491E4468CC
:102C3000E302F4D5C4F31303436043681A434260CC
:102C4000084630BC7047FEE74FF4001C1CEB410FF8
:102C500094BF1CEB430F09E041EA030C50EA4C0C13
:102C600052EA0C0C03D2994208BF9042704714BF3D
:102C70008B4282427047FEE74FF4001C1CEB410F71
:102C800094BF1CEB430F09E041EA030C50EA4C0CE3
:102C900052EA0C0C03D28B4208BF8242704714BF29
:102CA000994290427047FEE770B504460D46606851
:102CB000C0F30A5040F2FF71884207D160680003F8
:102CC00004BF2068002817D0022070BD20B920461C
:102CD000FFF797FF012866DA012D0FDB40F2FF7145
:102CE000091A8D420AD36068002847BF00202F4987
:102CF00000202F49C4E90001012070BD4142A942D2
:102D0000616806DA6FF31E51401941EA00506060B5
:102D100040E0401E63684519012205F1350062F369
:102D20001F53352801F00041636003D36160002028
:102D3000206070BD002015F11F0F04DA20682360A9
:102D40000022203562606A4212D0401E2568804110
:102D5000C2F12003C0439D4045EAD07025686668F3
:102D6000D54006FA03F32B4323606368D3406360C6
:102D700062680A43B0F1004F626003D80DD1207839
:102D8000C0070AD52068401C2060206828B9606808
:102D9000401C60604FF0FF3070BD6068884204BF27
:102DA00020680028F6D1002070BD00BF0000F0FFB1
:102DB0000000F07FF446400D40EAC120490006D2F1
:102DC00000F014F8004248BF6FF00040604700F088
:102DD0000DF84FF0004188428CBF084640426047E2
:102DE000400D40EAC120490080F00D8040F00040D5
:102DF000490DA1F58061491C05D4D1F11F0154BFD3
:102E0000C840C01770474FF000007047010040F104
:102E10000980F446404200F005F851F00041604757
:102E2000010000BF09D0B0FA80F18840C91CC1F58B
:102E30008461090501EBD02140057047F0B44FF0E3
:102E4000004591EA030F44BF6B4000F0BDBA00BFDC
:102E5000841A71EB030604D26E40001BB1411219B3
:102E600073414FF4001C1CEB410F34BF7CEB430655
:102E700084E00C0DA4EB1356362E7DDC012E43DCD2
:102E800045EAC32343EA525312BFD20292025B08BF
:102E9000240545EAC12141EA5051D2EBC0209941B5
:102EA00025D407D1B0FA80F610FA06F164D00020DC
:102EB000203608E0B1FA81F6B140C6F1200220FACE
:102EC00002F21143B0404FEAF474B4EB465434F0CC
:102ED00001064FEA74040AD8D6F50016760D04F000
:102EE0000044F04061FA06F25040F1404840C00A08
:102EF00040EA415021F0004128BF5FEA500550F1FF
:102F0000000044EBD12137E045EAC323DB0A45EA60
:102F1000C121C90AB6F120050EDD42EA0242120CB7
:102F2000C5F1200603FA06F6EB4042EA06056D42BB
:102F3000984161F100010DE062FA06F5F24055405A
:102F400063FA06FC82EA0C02F3405A406D4290415B
:102F500061EB030111F4801F05D1641E620502D0EC
:102F60006D004041494121F48011430875F100434F
:102F700050F1000041EB0451F0BC70471CEB410FD5
:102F800015D223F0004352EA43060BD04FEA4C0C13
:102F9000BCEB410F04D80C0D661E342EB7DDEBE7F9
:102FA000801A994150EA410608BF0021E4E708BFB2
:102FB0001CEB430F28BF6FF00001DDE7B0B581EADD
:102FC000030C0CF0004C40F2FF7515EA11541DBFC4
:102FD00015EA1357AC42AF4239E0E41923EA4553EE
:102FE00043F48013C90241F0004141EA505EC70238
:102FF0001100A7FB020200284FF00000EEFB0120A9
:103000004FF00001E3FB072118BF42F00102401816
:1030100000214941E3FB0E01A4F580640F0302D2B5
:1030200052004041494154F101046CDD470872F1FE
:10303000004250F1000051EB0451A1F580115CBF3A
:1030400041EA0C01B0BD4CEA05510020B0BD05EAD3
:103050001357AC4214BFAF4241E050EA410E1CBFCF
:1030600052EA430E02E061460020B0BD24423C44D7
:103070001BD15FEA070EF6D0090302BF014600200C
:10308000AEF1140EB1FA81F7AEEB070401FA07FEB8
:103090000C37C7F1200100FA07F7C8404EEA000ECE
:1030A00023EA455343F48013A2E733F00043B3FA15
:1030B00083F704BFB2FA82FE77440B3FE41BB7F1FB
:1030C000200E2FBF02FA0EF3BB40C7F1200E22FAEA
:1030D0000EFE38BF43EA0E03BA40641C82E750EA92
:1030E000410E14BF52EA430E6FF000014FF4001777
:1030F00017EB430F8ABF194617EB410FB5E74CEAB0
:1031000005510020B0BDD4F10104B4F120070FDA5D
:10311000C4F12007520828BF42F0010210FA07F557
:1031200001FA07F7E1BF2A43E0403843E1400FE0EE
:10313000352C98DCC7F1200452EA400220FA07F24D
:1031400018BF42F0010231FA07F0A1400A43002102
:1031500072F1004250F1000051EB0C01B0BDFEE7EE
:103160002DE9F04140F2FF7581EA030C0CF0004CB0
:1031700015EA11541DBF15EA1357AC42AF42E9E0FE
:10318000BC41C1F31301C3F31303801A994143F403
:10319000801304D2641E4000494180185941C9027D
:1031A00041EA5051B1FBF3F603FB1611A2FB067581
:1031B000D7EBC020A94102D2761E80185941C9021E
:1031C00041EA5051B1FBF3FE03FB1E11A2FB0E7549
:1031D000D7EBC020A94103D2AEF1010E80185941AE
:1031E000890241EA9051760546EA8E2EB1FBF3F64C
:1031F00003FB1611A2FB0675D7EB8020A94102D272
:10320000761E80185941C90241EA50514EEA060E15
:10321000B1FBF3F603FB1611A2FB0675D7EBC0203A
:10322000A94102D2761E80185941C90241EA505183
:10323000B1FBF3F703FB1711A2FB0735D3EBC0205B
:10324000A94167F100070CBF004247F0010766F390
:10325000D5274FEA1E31B80814F5806414DDBD0788
:1032600075F1004250EB0E5051EB045111F5801FE7
:103270005CBF41EA0C01BDE8F0814CF07F6141F098
:10328000E0410020BDE8F081BD076D0840EA0E5026
:1032900041F48011D4F10104B4F120060ADAC4F13A
:1032A00020060200E04001FA06F3E1401843B24074
:1032B00015430EE0342C14DCC6F1200445EA400529
:1032C0006D0820FA06F2154321FA06F0A1400D43DD
:1032D000002175F1004250F1000051EB0C01BDE8F6
:1032E000F08100205FEA0C01BDE8F081CFB99218AF
:1032F0005B41B3FA83F704BFB2FA82F6BF190B3F02
:10330000B7F120062FBF02FA06F3BB40C7F1200633
:1033100022FA06F638BF3343BA401CB1E419641EE2
:103320002FE77F4231F00041B1FA81F404BFB0FAD7
:1033300080F6A4190B3CB4F120062FBF00FA06F169
:10334000A140C4F1200620FA06F638BF3143A04060
:103350003C1B16E7AC421ABF05EA1357AF4214E014
:1033600050EA41061CBF52EA4306BFE750EA410754
:10337000304661461CBF41EA0551BDE8F08152EA82
:10338000430C08BFC143BDE8F08100204FF4001694
:1033900016EB410F98BF16EB430F08BF16EB410F1A
:1033A00024BFC14305E016EB430F0CBF61464CEA56
:1033B0000551BDE8F08191FBF2F303FB1211C0E966
:1033C000003170477047FEE7841A71EB030603D2A1
:1033D000001BB141121973414FF4001C1CEB410F4B
:1033E00034BF7CEB430443E00C0DA4EB1356352EA5
:1033F00050DC45EAC323DB0A45EAC121C912B6F114
:1034000020050DDD63FA05F6EB4086EA030512425E
:1034100018BF45F00105C01851F100010CD213E0AE
:1034200062FA06F5F2405540F3415A40B340F3408A
:103430005A408018594107D349085FEA30005FEAD3
:10344000350528BF45F0010501F58011420875F1E9
:10345000004250F1000041EB0451F0BC4FF4001C5D
:103460001CEB410F38BF70470020090D090570475C
:103470001CEB410F10D252EA43060BD0BCEB410FBC
:1034800005D80C0DAB43661E342EB5DD02E0AB4310
:1034900080185941F0BC7047F0BC7047002203E02F
:1034A0000B788354491C521C0B78002BF8D1100068
:1034B00070470120DFF88C190860DFF88C09DFF80D
:1034C0008C190860DFF8880900684007FAD54FF4C6
:1034D0008170DFF8801908605FF08070DFF878197C
:1034E00008605FF04070DFF8741908604FF4827074
:1034F000DFF86C190860DFF8580900688007FAD512
:103500004FF48370DFF84C190860FF20DFF854197E
:103510000860EF20DFF8501908604AF6AA00DFF8CB
:103520004C1908600220DFF8481908604FF4FC606D
:10353000DFF8401908604FF46070DFF83C1908604C
:103540004FF40070DFF8341908605FF4A820DFF84A
:10355000301908604FF40050DFF8281908605FF058
:103560008860DFF8241908608C20DFF820190860D3
:103570008C20DFF81C1908608C20DFF8181908600F
:1035800048F2A000DFF8101908600320DFF80C19DA
:1035900008600F20DFF8081908600420DFF804191C
:1035A00008605FF48030DFF8001908605FF0E030F9
:1035B000DFF8F8180860DFF8F808DFF8F818086096
:1035C0005FF0E030DFF8F0180860DFF8F008DFF8AF
:1035D000F01808605FF0E030DFF8E81808605FF08E
:1035E000E030DFF8E41808605FF0E030DFF8DC1866
:1035F00008605FF0E030DFF8D8180860704700001E
:1036000080B5FFF756FF00F09BFC00F0C7FEFEF709
:1036100089F9FEF765F900F0F1FE4FF4FA7000F059
:103620004FFEDFF8B0080078C006FAD500BF00F002
:103630005FFE0320DFF838180860DFF840080068F4
:10364000DFF894180840DFF834180860012000F013
:1036500043FEDFF8800800788006FAD500220021BA
:103660005120FEF789F8012000F036FEDFF86408EB
:1036700000788006FAD5002203214020FEF77CF86E
:10368000012000F029FEDFF84C0800788006FAD50A
:10369000002200217520FEF76FF8012000F01CFECB
:1036A000DFF8300800788006FAD50022FF210020DC
:1036B000FEF762F8012000F00FFEDFF8180800782E
:1036C0008006FAD5002200211020FEF755F80120CF
:1036D00000F002FEDFF8FC0700788006FAD5002231
:1036E000FF210120FEF748F8012000F0F5FDDFF88A
:1036F000E40700788006FAD5002200211120FEF7A9
:103700003BF8022000F0E8FDDFF8C80700788006EB
:10371000FAD5DFF8800700684FF6FB710840DFF844
:103720007417086001220A21DFF8B007FEF7B6F827
:10373000DFF86007006850F00C00DFF858170860E9
:10374000012000F0C9FDDFF88C0700788006FAD56B
:10375000DFF8400700684FF6F7710840DFF83417CC
:10376000086001220A21DFF87807FEF797F8DFF8F2
:103770002407006850F00C00DFF8181708600220DA
:1037800000F0AAFDDFF84C0700788006FAD5DFF8D4
:10379000EC0600684FF6F071084050F48070DFF8D6
:1037A000DC160860C82000F097FDDFF828070078D5
:1037B0008006FAD500226E210020FDF7DDFF6E2085
:1037C000DFF820170870012000F086FD00226E212E
:1037D0000120FDF7D1FF6E20DFF80C170870DFF82D
:1037E000F40600788006FAD5002200211020FDF7AB
:1037F000C3FF012000F070FDDFF8D80600788006D6
:10380000FAD5012000F068FDDFF8C80600788006D0
:10381000FAD5002200211120FDF7AEFF0A2000F0AA
:103820005BFDDFF8B00600788006FAD5322000F0A4
:103830003BFD07E00020DFF8B4160860192000F017
:1038400033FD00BF4AF6AA20DFF8A4160860DFF8AF
:1038500084060078C00714D5DFF83806006890F0B9
:103860008000DFF830160860DFF8280600680006E0
:1038700003D5642000F00CFD03E040F26C7000F012
:1038800007FDDFF87006006810F0204F11D0DFF858
:103890000406006850F08000DFF8F8150860642026
:1038A00000F0F6FC0120FCF719FC0020DFF84416BC
:1038B0000860DFF844064088002800F0DF81DFF868
:1038C000D405006850F08000DFF8C8150860642057
:1038D00000F0DEFCDFF824064078202869D1DFF80C
:1038E0001C06807FDFF818160978884261D000BF77
:1038F000012007E0DFF804160144C979DFF8042647
:103900001154401C0B28F5D3DFF8880500684FF6EA
:10391000FB710840DFF87C15086001220A21DFF8FE
:10392000BC05FDF7BBFFDFF86C05006850F00C002C
:10393000DFF860150860012007E0DFF8C0150144DA
:10394000C97CDFF8C4251154401C0B28F5D3DFF8DF
:10395000440500684FF6F7710840DFF83815086035
:1039600001220A21DFF87805FDF798FFDFF824052A
:10397000006850F00C00DFF81C1508600022DFF82A
:103980007C050079012801D14FF48072DFF86C05C5
:103990004079012801D152F08002DFF8E00400688C
:1039A00010F4CC600243DFF85405807FDFF8501537
:1039B0000870DFF848054078152840F05C81DFF892
:1039C0003C050078AA2809D1DFF84015DFF840054A
:1039D000FFF764FDDFF83C15086008E0DFF83815F4
:1039E000DFF82C05FFF75AFDDFF828150860DFF82F
:1039F000A40400684FF6FB710840DFF898140860D3
:103A00000121DFF80005FDF75BFFDFF8880400689F
:103A100050F00C00DFF87C1408600022002005E064
:103A2000DFF8F81431F810108A18401C0428F7D376
:103A30009208CEA1DFF8D804DFF8D8341B68184408
:103A4000FEF7D0F8DFF8CC1409684018DFF8C4148A
:103A500008600022002005E0DFF8C41431F81010DF
:103A60008A18401C0428F7D39208C0A1DFF8A004EC
:103A7000DFF8A0341B681844FEF7B4F8DFF894149C
:103A800009684018DFF88C1408600022002005E067
:103A9000DFF8901431F810108A18401C0428F7D36E
:103AA0009208B2A1DFF86804DFF868341B68184494
:103AB000FEF798F8DFF85C1409684018DFF8541432
:103AC00008600022002005E0DFF85C1431F81010D7
:103AD0008A18401C0428F7D39208A4A1DFF8300408
:103AE000DFF830341B681844FEF77CF8DFF8241444
:103AF00009684018DFF81C1408600022002005E067
:103B0000DFF8281431F810108A18401C0428F7D365
:103B1000920896A1DFF8F803DFF8F8331B68184421
:103B2000FEF760F8DFF8EC1309684018DFF8E413DB
:103B30000860002292088DA1DFF8D403DFF8D433A7
:103B40001B681844FEF74EF8DFF8C81309684018E0
:103B5000DFF8C01308600022002005E0DFF8D01372
:103B600031F810108A18401C0428F7D392087FA15E
:103B7000DFF89C03DFF89C331B681844FEF732F82B
:103B8000DFF8901309684018DFF8881308600022F6
:103B9000002005E0DFF89C1331F810108A18401C53
:103BA0000428F7D3920871A1DFF86403DFF86433C7
:103BB0001B681844FEF716F8DFF858130968401818
:103BC000DFF850130860DFF83C03027867A1DFF8E4
:103BD0004003DFF840331B681844FEF703F8CD4973
:103BE00009684018CB490860AA4800684FF6F77189
:103BF0000840A84908600121C348FDF761FEA548B7
:103C0000006850F00C00A3490860BF48027857A133
:103C1000BF48C04B1B681844FDF7E4FFBD49096865
:103C20004018BC490860B6480278C349B848B94B47
:103C30001B681844FDF7D6FFB64909684018B54916
:103C40000860B44800680105090DB148FDF78BFE16
:103C5000020092B2B949AE48AE4B1B681844FDF75A
:103C6000C1FFAC480068801DAA490860A9480168E6
:103C7000A748FDF70DFF00209F4908609548007890
:103C800000077FF5DEAD9948006800280ED00228B5
:103C90003CD023D304286BD050D3062800F0988062
:103CA000C0F07E80072800F0AB80C0E0032208E06F
:103CB0009E4800EB420030F8020C9C4921F81200AB
:103CC000521E002AF4D1002000F0A4FB0005000DD4
:103CD00096490880012000F095FBA8E0032208E047
:103CE000934800EB420030F8020C914921F8120091
:103CF000521E002AF4D1072000F08CFB0005000DB5
:103D00008B490880022000F07DFB90E0032208E050
:103D1000854800EB420030F8020C834921F812007C
:103D2000521E002AF4D1022000F074FB0005000DA1
:103D30007D490880032000F065FB78E0032208E05D
:103D4000774800EB420030F8020C754921F8120068
:103D5000521E002AF4D1032000F05CFB0005000D88
:103D60006F490880042000F04DFB60E025752300BA
:103D7000032208E06F4800EB420030F8020C6D4966
:103D800021F81200521E002AF4D1042000F042FB58
:103D90000005000D67490880052000F033FB46E070
:103DA000032208E05F4800EB420030F8020C5D4956
:103DB00021F81200521E002AF4D1052000F02AFB3F
:103DC0000005000D57490880062000F01BFB2EE07F
:103DD000032208E0514800EB420030F8020C4F4942
:103DE00021F81200521E002AF4D1062000F012FB26
:103DF0000005000D49490880072000F003FB16E08C
:103E0000032208E04A4800EB420030F8020C48491F
:103E100021F81200521E002AF4D1072000F0FAFA0D
:103E20000005000D42490880002000F0EBFA2F4801
:103E300000680728BFF4FEAC2C480068401C2B49E2
:103E40000860FBE408000240F860E2231C00024026
:103E5000000002400C000240240002402800024002
:103E6000040002400C800A4004800A4018800A4086
:103E700000800A400C000B4004000B4000000B4087
:103E800018000B4008000B4010000B400C800C4049
:103E900004800C4000800C4018800C400C800E40C8
:103EA00008800E4018800E4010800E4000E400E0B4
:103EB000E0E0404004E400E008E400E0E0E020E06E
:103EC0000CE400E010E400E014E400E018E400E09A
:103ED0001CE400E018000020E0FDFFFF01000020CE
:103EE0000D0000201D0000201E000020F001002019
:103EF0000080064000020020FC0100202801002074
:103F00001C000020000000200C0000207847000862
:103F1000100A0020EC01002080470008B0010020BA
:103F200098010020A80100209001002088010020B5
:103F3000B8010020A0010020684700087047000871
:103F40000120DFF8D81308604FF4FA50DFF8D013DF
:103F500008600120DFF8CC1308600020DFF8C813E8
:103F600008604FF48040DFF8C41308600920DFF8D0
:103F7000C0130860704780B5DFF8B80300680028F8
:103F800013D0DFF8B0030068401EDFF8A813086004
:103F9000DFF8A0030068002807D1DFF89C03006861
:103FA00050F00100DFF890130860DFF8900300681C
:103FB000002876D0DFF884030068401EDFF87C1309
:103FC0000860DFF87803006800286AD1DFF868032A
:103FD000006850F00200DFF8601308600FE0DFF8BF
:103FE00060030068DFF85C13DFF85C231268885414
:103FF000DFF854030088401CDFF84C130880DFF81A
:104000004C030068C00605D4DFF83C030068B0F537
:10401000847FE4D3DFF830030088022809DBDFF86F
:1040200024030078AA2809D0DFF818030078BB28F9
:1040300004D00020DFF81013086032E0DFF804033A
:104040004078152805D14FF48040DFF8FC124880F5
:1040500027E0DFF8F002407820281ED14FF480508E
:10406000DFF8E4124880DFF8E0020188DFF8D402CC
:10407000FDF779FCDFF8D8120880DFF8D402008859
:10408000002805D14FF40040DFF8BC12488008E05A
:104090000020DFF8B412086003E00020DFF8A81267
:1040A0000860DFF8B0020068002851D0DFF8A402F1
:1040B0000068401EDFF89C120860DFF89802006874
:1040C000002845D1DFF87002006850F00400DFF8E6
:1040D000681208600FE0DFF880020068DFF87C12E9
:1040E000DFF87C2212688854DFF874020088401CD4
:1040F000DFF86C120880DFF86C020068C00604D498
:1041000097480068B0F5847FE5D395480088042877
:1041100003DA0020924908601AE04FF48050904979
:1041200048808F4801888D48FDF71DFC8E49088026
:104130008D480088002808D188480078022804D1DA
:104140004FF400408649488002E00020844908601E
:104150008648006800280ED084480068401E8349C5
:10416000086082480068002805D17348006850F054
:104170000800714908607E48006800280ED07C481D
:104180000068401E7A49086079480068002805D117
:104190006948006850F01000674908607548006879
:1041A00000280ED073480068401E724908607148AC
:1041B0000068002805D16048006850F020005E4982
:1041C00008606D48006800280ED06B480068401EEB
:1041D0006949086068480068002805D156480068A9
:1041E00050F02000544908606448006800280ED050
:1041F00062480068401E6149086060480068002805
:1042000005D14D48006850F080004B4908605C487B
:10421000006800280ED05A480068401E58490860BF
:1042200057480068002805D14348006850F4807062
:10423000414908605348006800280ED05148006882
:10424000401E504908604F480068002805D13A4890
:10425000006850F40070384908604B480068002836
:104260000ED049480068401E47490860464800682B
:10427000002805D13048006850F480602E4908605D
:104280000020294908604FF480404049086001BD82
:1042900072B628490860284800684008400026494E
:1042A000086062B67047000072B630490860224864
:1042B000006830F008002049086062B670470000CE
:1042C00072B62B4908601C48006830F010001A498B
:1042D000086062B67047000072B62649086016484A
:1042E000006830F020001449086062B67047000092
:1042F0004CF6CC402649086045F2555024490860E8
:10430000032024490860244800680028FBD14AF6AD
:10431000AA201F4908607047000000000400074001
:1043200008000740580007405400074000E100E043
:104330000C000740C001002018000020C40100202C
:104340000000034028010020FC0100201800034069
:10435000F4010020C801002000800340200000205C
:104360000002002018800340F8010020CC0100204A
:10437000D0010020D4010020D8010020DC01002061
:10438000E0010020E4010020E801002080E200E0DC
:1043900000800640048006400C8006405FF0FF303D
:1043A0000D4908605FF0FF300C4908600C480D496A
:1043B00048620D480B4948600C480A4988620B481E
:1043C0000849886007480A490860012009490860CF
:1043D000E1200949086070472C800240208002409B
:1043E000008003400004002000000340000034C0AF
:1043F000088002404C800240048002400E480F4971
:1044000008607047000110F4F8700B4908430B492D
:1044100008607047000110F4F8700749084350F035
:10442000020006490860054800688007FBD404487C
:1044300000680005000D7047011000020080084070
:104440001880084000C1814001C0804101C0804106
:1044500000C1814001C0804100C1814000C1814054
:1044600001C0804101C0804100C1814000C1814044
:1044700001C0804100C1814001C0804101C0804134
:1044800000C1814001C0804100C1814000C1814024
:1044900001C0804100C1814001C0804101C0804114
:1044A00000C1814000C1814001C0804101C0804104
:1044B00000C1814001C0804100C1814000C18140F4
:1044C00001C0804101C0804100C1814000C18140E4
:1044D00001C0804100C1814001C0804101C08041D4
:1044E00000C1814000C1814001C0804101C08041C4
:1044F00000C1814001C0804100C1814000C18140B4
:1045000001C0804100C1814001C0804101C08041A3
:1045100000C1814001C0804100C1814000C1814093
:1045200001C0804101C0804100C1814000C1814083
:1045300001C0804100C1814001C0804101C0804173
:1045400000C1814000C0C101C30302C2C60607C743
:1045500005C5C404CC0C0DCD0FCFCE0E0ACACB0BB3
:10456000C90908C8D81819D91BDBDA1A1EDEDF1FE3
:10457000DD1D1CDC14D4D515D71716D6D21213D3D3
:1045800011D1D010F03031F133F3F23236F6F73783
:10459000F53534F43CFCFD3DFF3F3EFEFA3A3BFB73
:1045A00039F9F83828E8E929EB2B2AEAEE2E2FEF23
:1045B0002DEDEC2CE42425E527E7E62622E2E32393
:1045C000E12120E0A06061A163A3A26266A6A767C3
:1045D000A56564A46CACAD6DAF6F6EAEAA6A6BAB33
:1045E00069A9A86878B8B979BB7B7ABABE7E7FBF63
:1045F0007DBDBC7CB47475B577B7B67672B2B37353
:10460000B17170B050909151935352929656579702
:10461000559594549C5C5D9D5F9F9E5E5A9A9B5BF2
:1046200099595898884849894B8B8A4A4E8E8F4FA2
:104630008D4D4C8C44848545874746868242438312
:104640004181804019E050F8041BCB0744BFA9F119
:1046500001035918121F0023042A41F8043BF9D220
:104660005FEA827C0B4604D54FF0000CA1F800C035
:104670009B1CD10744BF0021197050F8042B002A5D
:10468000E1D1704710B450F8041B79B10268436857
:1046900002440830DC0744BFA9F10104E31852F8D2
:1046A000044B43F8044B091FF9D1ECE710BC7047E9
:1046B00010B5074979441831064C7C44163404E09F
:1046C0000A68081D114488470146A142F8D110BD6F
:1046D00008000000280000006DFFFFFFE40100005B
:1046E00020000020000000009DFFFFFF20000000D0
:1046F000D800000000000020000000000120C0469B
:10470000002801D0FFF7D4FF0020AFF30080FEF7B0
:1047100077FF00F000F800F001B8FEE707463846E2
:1047200000F002F8FBE7FEE72021090326311820FC
:10473000ABBEF9E7762E312E352030342E30352EB3
:10474000323032330000000002485FF00061016047
:10475000704700BF08ED00E080B5FFF7F5FFAFF34D
:104760000080FFF7CBFF01BD257523454E440000B7
:10477000252E34580D0A0000374731230000000071
:104780003747322300000000CECECE20C8D0C7006D
:1047900041524D5F4D3300006D6F642030000000CA
:1047A000524D2000FEE7FEE7FEE7FEE7FEE7FEE7EC
:1047B000FEE7FEE7FEE7FEE7FEE7FEE7FEE7FEE7D1
:1047C000FEE7FEE7FEE7FEE7000400400200F91303
:1047D000B90A0000000400400200FF13B90A0000FB
:0847E000FFFFFFFFFFFFFF00D8
:04000005080047594F
:00000001FF
